:1000000000308A0018280000243084008313000880
:10001000031917280230F800F701F70B0D28F80B29
:100020000C289730F700F70B1328800B0A280800DC
:10003000840183131F308305713083168F000F08EE
:10004000061383120617831603170908C03989009F
:1000500003131F129F1200300317880083128701B9
:1000600088018901FF300313A000A3018316031741
:100070000908C039890003131F129F1201300317AA
:100080008800831203131F139F1783169F17831271
:100090001F149412A01220088316870083122016C2
:1000A0002008831687008312A0112008831687007A
:1000B0000130831294000030831694000108C73980
:1000C00028388100831290010030F8000438920033
:1000D000FF308316920083122011200883168700B8
:1000E00083120711831609130C30831297008316AD
:1000F0009B019C0101309D008312A01020088316F3
:100100008700831287100C309D0001308000031798
:100110008701880189017130831603138F000F084E
:10012000831295019B013C30A1000430F8001F08A8
:10013000C33978049F004230F700F70B9D28000078
:100140009F149F18A12883161E088312A20022085C
:100150002102031CB0282308953C0318A30AB328E6
:10016000A308031DA3032308950023089B00201365
:10017000200883168700831207136430A40004202C
:100180002013200883168700831207176430A40009
:0601900004209528630025
:04400E00F52CFF3F4F
:00000001FF
